:0200000480007A
:100000006F00C004732F2034930F8000630AFF0336
:10001000930F90006306FF03930FB0006302FF038A
:10002000170F0080130F0FFE63040F0067000F000F
:10003000732F203463540F006F004000136E9E53E3
:10004000171F00002320CFFD6FF09FFF732540F1A5
:100050006310050073251030635805000F00F00F82
:10006000130E100073000000130E00009702000032
:10007000938282F973905230735020307350303035
:1000800073504030970200809382C2F7638C020065
:10009000739052109302B01A739022307323203061
:1000A000E39E62F873500030970200009382420191
:1000B00073901234732540F173002030130E20002A
:1000C000930000001301100063E620006312C02FAC
:1000D0006316C001E3EE20FE631CC02D130E30003A
:1000E0009300E0FF1301F0FF63E620006312C02DD0
:1000F0006316C001E3EE20FE631CC02B130E40000C
:10010000930000001301F0FF63E620006312C02B90
:100110006316C001E3EE20FE631CC029130E5000DD
:10012000930010001301000063E420006314C00179
:100130006310C029E3EE20FE130E60009300F0FF71
:100140001301E0FF63E420006314C0016312C027C1
:10015000E3EE20FE130E70009300F0FF1301000089
:1001600063E420006314C0016314C025E3EE20FEA5
:10017000130E8000B7000080370100801301F1FFEB
:1001800063E420006314C0016314C023E3EE20FE87
:10019000130E900013020000B70000F0370100F0CA
:1001A0001301F1FF63E620201302120093022000E6
:1001B000E31452FE130EA00013020000B70000F07B
:1001C000370100F01301F1FF1300000063E2201E6D
:1001D0001302120093022000E31252FE130EB0002D
:1001E00013020000B70000F0370100F01301F1FF27
:1001F000130000001300000063EC201A1302120029
:1002000093022000E31052FE130EC0001302000000
:10021000B70000F013000000370100F01301F1FFF8
:1002200063E820181302120093022000E31252FE2A
:10023000130ED00013020000B70000F013000000FE
:10024000370100F01301F1FF1300000063E22016F4
:100250001302120093022000E31052FE130EE0007E
:1002600013020000B70000F01300000013000000AC
:10027000370100F01301F1FF63EC201213021200AA
:1002800093022000E31052FE130EF0001302000050
:10029000B70000F0370100F01301F1FF63EA20100E
:1002A0001302120093022000E31452FE130E000109
:1002B00013020000B70000F0370100F01301F1FF56
:1002C0001300000063E6200E1302120093022000C8
:1002D000E31252FE130E100113020000B70000F0EB
:1002E000370100F01301F1FF1300000013000000BC
:1002F00063E0200C1302120093022000E31052FE70
:10030000130E200113020000B70000F013000000DC
:10031000370100F01301F1FF63EC20081302120013
:1003200093022000E31252FE130E3001130200006C
:10033000B70000F013000000370100F01301F1FFD7
:100340001300000063E6200613021200930220004F
:10035000E31052FE130E400113020000B70000F03C
:100360001300000013000000370100F01301F1FF3B
:1003700063E020041302120093022000E31052FEF7
:1003800093001000636A10009380100093801000A7
:1003900093801000938010009380100093801000D1
:1003A000930E3000130E50016394D001631CC00102
:1003B0000F00F00F63000E00131E1E00136E1E00D0
:1003C000730000000F00F00F130E10007300000008
:1003D000731000C0000000000000000000000000DA
:1003E000000000000000000000000000000000000D
:1003F00000000000000000000000000000000000FD
:0404000000000000F8
:1010000000000000000000000000000000000000E0
:1010100000000000000000000000000000000000D0
:1010200000000000000000000000000000000000C0
:1010300000000000000000000000000000000000B0
:081040000000000000000000A8
:040000058000200057
:00000001FF
